:0A00000075817F7401F58F02000E78
:10000B00021566C209C207C208C20AC20BC20CC2E1
:10001B000DC20EC20FC206755200756500756600E3
:10002B00C200C201C202756700756800756900F5F0
:10003B006A756B00756C00C203C204C2057557006C
:10004B00755100C211C212C213C21475430075441C
:10005B0000754500754600754700754800754900E9
:10006B00754A00754B00754C00757100C218C219AA
:10007B00C21AC21BC21CC21DC21EC21FC220C22179
:10008B00C222C223C224C225D2267530007531008C
:10009B0075320075330075340075350074009000AF
:1000AB0010F0900011F0900012F0900013F09000FF
:1000BB0014F0740090001DF0740090003CF01208D6
:1000CB007A1208AF755DFF755EFF755FFF120C004E
:1000DB001215431202811202811202811202811245
:1000EB0001B9120281120281120281120281121CC9
:1000FB0019121C39121BCED219D217301206121537
:10010B008B020106301A061219600201061215DC69
:10011B001219B912087A1208AF120C42120C5420A1
:10012B001021120C6A120CAF20160F120C96120C27
:10013B00C1120CD3120CEC02014B12193A12194ECC
:10014B00120C00120C801212D01211E11211751246
:10015B00149E121899120D37120D72120DD7120D23
:10016B00C6120E1112134E120D05120D1720190681
:10017B0020030D0201AE30172CC2171218C4C2197E
:10018B00C203C205856768A20092018565661212DB
:10019B00BC12052312044212046F12049C1204C9F0
:1001AB000201B0D21712110F12108D020106E55F7A
:1001BB00C2E1F55F120C00120281E55FD2E1C2E2EF
:1001CB00F55F120C00120281E55FD2E2C2E3F55F2C
:1001DB00120C00120281E55FD2E3C2E4F55F120C50
:1001EB0000120281E55FD2E4C2E5F55F120C00124A
:1001FB000281E55FD2E5F55F120C00120281E55F2B
:10020B00C2E6D2E0F55FE55DC2E3F55D120C007F5F
:10021B000F120281DFFBE55FD2E6D2E0C2E5F55FAC
:10022B00120C00120281E55FD2E5C2E4F55F120CFD
:10023B0000120281E55FD2E4C2E3F55F120C0012FB
:10024B000281E55FD2E3C2E2F55F120C001202817C
:10025B00E55FD2E2C2E1F55F120C00120281E55FAD
:10026B00D2E1F55F120C0012028122783279FF0085
:10027B0000D9FCD8F822784B79FF0000D9FCD8F8CC
:10028B002278967996D9FED8FA22E627F525080921
:10029B00E637F526782522C3E697F5250809E69774
:1002AB00F526782522862587270809862687281292
:1002BB000335782A22862A08862B08862C08862D59
:1002CB0087270987281202D87825792C22752E00CA
:1002DB00752F1012031A1202EB12030ED52FF422F4
:1002EB00C3E52C9527E52D9528E52E94005001228A
:1002FB00E52C9527F52CE52D9528F52DE52E94006D
:10030B00F52E22B3E52533F525E52633F52622C355
:10031B00E52A33F52AE52B33F52BE52C33F52CE5C4
:10032B002D33F52DE52E33F52E22E5258527F0A46B
:10033B00F52A85F02BE5268528F0A4F52C85F02DE4
:10034B00E5268527F0A4252BF52BE52C35F0F52C90
:10035B00E52D3400F52DE5258528F0A4252BF52B6F
:10036B00E52C35F0F52CE52D3400F52D22E582C476
:10037B00540FF9E583C469227A0FC2A0D293A292DB
:10038B0033C933C9C293DAF2F8D2A022D2A07A05CC
:10039B0074E0C293C2A0339294D293DAF512038322
:1003AB00883C893D533D0F22D2A07A0574E8C29355
:1003BB00C2A0339294D293DAF5120383883A893B25
:1003CB00533B0F22D2A07A0574F0C293C2A0339292
:1003DB0094D293DAF51203838838893953390F2273
:1003EB00D2A07A0574F8C293C2A0339294D293DA56
:1003FB00F51203838836893753370F221203B375EF
:10040B00320075330078307534117535007934123C
:10041B000295863008863175320075330078307559
:10042B0034E875350379341202B07534F2753586BC
:10043B0079341202C0E622A847A948D297D2A1D29A
:10044B0095E944707A08C2A3C2A2339296D2A3DA7A
:10045B00F57A08E8C2A3C2A2339296D2A3DAF5C208
:10046B0097D2A222A849A94AD297D2A1D295E94400
:10047B00F07A08C2A3C2A2339296D2A3DAF57A0815
:10048B00E8C2A3C2A2339296D2A3DAF5C297D2A244
:10049B0022A845A946D297D2A2D295E944707A08F0
:1004AB00C2A3C2A1339296D2A3DAF57A08E8C2A30B
:1004BB00C2A1339296D2A3DAF5C297D2A122A84356
:1004CB00A944D297D2A2D295E944F07A08C2A3C22A
:1004DB00A1339296D2A3DAF57A08E8C2A3C2A1336C
:1004EB009296D2A3DAF5C297D2A122A84BA94CD2ED
:1004FB0097D2A2D2A1E944707A08C2A3C2953392D3
:10050B0096D2A3DAF57A08E8C2A3C295339296D2B3
:10051B00A3DAF5C297D29522E56320E0041205D445
:10052B002230E3041205D4221205D422E56320E025
:10053B00041206352230E304120635221206352248
:10054B00740090001DF090001E12064E853E301276
:10055B00066D1206DD858243858344740190001D70
:10056B00F090001F12064E853F3012066D1206DD0D
:10057B00858245858346740290001DF09000201201
:10058B00064E85403012066D1206DD858247858347
:10059B0048740390001DF090002112064E854130E7
:1005AB0012066D1206DD85824985834A22740490FA
:1005BB00001DF090002212064E85423012066D127D
:1005CB0006DD85824B85834C22740090001DF090D4
:1005DB00001E12064E853E3012066D8582438583C2
:1005EB0044740190001DF090001F12064E853F30A1
:1005FB0012066D858245858346740290001DF0902E
:08060B00002012064E8540306C
:1006130012066D858247858348740390001DF09010
:10062300002112064E85413012066D85824985836D
:100633004A22740490001DF090002212064E854257
:100643003012066D85824B85834C22E0F53075317F
:10065300007532007533007830753457753501797C
:1006630034120295868208868322E530753100753F
:100673003200753300783070030206B48582348506
:10068300833579341202B075340A75350079341222
:1006930002C01216FCE0F534753500793412029568
:1006A30075340775350079341202A2868208868371
:1006B300221216FCE0B407030206C250027407F5C7
:1006C3003475350079341202957534077535007920
:1006D300341202A286820886832285823085833182
:1006E3007532007533007830853A34853B3579347B
:1006F300120295868208868322B402012240027484
:100703000022B40301224002740322B40F012240E9
:1007130002740022B40F01224002740F22E551B487
:100723000006E56CB4031022B40C06E56CB40707AD
:1007330022E56CB40B01224002740022E551B4009F
:1007430006E56CB4031022B40C06E56CB4070C2266
:10075300E56CB40B0B22400D74032240087407228E
:100763004003740B2222E551B40009E56CB405196A
:1007730002079022B40C09E56CB40D1702079A2204
:10078300E56CB415180207A42240027400F56C123C
:100793000F932240027400F56C120FAF22400274D3
:1007A30000F56C120FE322B403012240027400220D
:1007B300B40F01224002740F22B4100122400274CC
:1007C3000022B41001224002741022B4110122400D
:1007D30002740222B40102741122B45F01224002A6
:1007E300745F22B46001224002746022B42F01229C
:1007F3004002742F22B43001224002743022B40F1D
:1008030001224002740F22B4C00122400274C022AC
:10081300B4F00122400274F022B478012240027441
:100823007822C3B44701224002744722B40F012245
:100833004002740F22B40F01224002740022B40458
:1008430001224002740022B40401224002740422F3
:10085300B40501224002740522B410030208645057
:100863000022900010E004B410027400F090000025
:10087300A98229F582E022900014E0FA900011E0A9
:1008830004B40F0274FFF0900965932A900014F0EA
:10089300900013E004B410027400F0F9900014E027
:1008A300FA900000E58229F582EAF022900014E034
:1008B300FA900012E004B4110274FFF090097493EB
:1008C3002A900014F012089322120865540160085C
:1008D300120865541F246022747F2212086575F084
:1008E30020842212086575F010842212086575F0C1
:1008F3001F842212086575F02084F812086575F0CC
:100903003F842822120865540175F00CA4221208B2
:100913006575F0558475F00CA4221208F6C2E02226
:1009230012086575F0338475F003A490093273746B
:100933000222740422740522740722740922740BA0
:100943002212086575F0338475F003A4900953737C
:100953007402227403227405227407227408227419
:100963000A2203002C0C01057E2133E6FF0B4D68A0
:10097300146405140D004B1A26351E1A96114042B5
:0E098300C8C9464C414D452043484F524420C0
:100991004D414348494E45204D4F44554C45204516
:1009A10055524F205241434B2056455253494F4EC9
:1009B100202D20323031372056455253494F4E2099
:1009C100312E303420286329627920616D7065727F
:1009D100650004070C04070C10070C101300040732
:1009E100090407090C07090C100004070B04070B85
:1009F1000C070B0C100004060B04060B0C060B0C69
:100A0100100004080B04080B0C080B0C1000020466
:100A1100070204070C04070C0E0004050704050770
:100A21000C05070C100004070E04070C0E070C0E32
:100A310010000306090306090F06090F1200040737
:100A41000A04070A0C070A0C100004060A04060A25
:100A51000C060A0C100005070C05070C11070C11F8
:100A610013000205070205070C05070C0E00040B15
:100A71000E040B0E0C0B0E0C10000B10150B1015A9
:100A81000C10150C17000000000000000000000011
:100A9100000003070C03070C0F070C0F13000307DB
:100AA100090307090C07090C0F0003070A03070ACA
:100AB1000C070A0C0F0003060A03060A0C060A0CAF
:100AC1000F0003080A03080A0C080A0C0F000203AE
:100AD100070203070C03070C0E00030507030507B4
:100AE1000C05070C0F0003070E03070C0E070C0E75
:100AF1000F000306090306090C06090C0F00040880
:100B01000C04080C10080C10140004080A04080A4C
:100B11000C080A0C100002070C02070C0E070C0E41
:100B2100130005070A05070A0C070A0C1100050A3C
:100B31000C050A0C110A0C11160003070B03070B15
:100B41000C070B0C0F000000000000000000000C5F
:100B51000C0004070C6300040709630004070B631E
:100B61000004060B630004080B6300020407630022
:100B7100040507630004070E630003060C63000409
:100B8100070A630004060A630005070C63000205F7
:100B910007630002050A63000C18246301020304C1
:100BA10005060708090A0B630003070C6300030726
:100BB10009630003070A630003060A630003080AC6
:100BC10063000203076300030507630003070E6365
:100BD10000030609630004080C630004080A6300AB
:100BE10002070C630005070A6300050A0C6300187D
:100BF1003048630102030405060708090A0B63C2B2
:100C0100B4C2B1C2B7C2B3E55D7F083392B5D2B306
:100C1100C2B3DFF7B2B40000C2B4E55E7908339223
:100C2100B5C2B3D2B3D9F7D2B10000C2B1E55F7991
:100C3100083392B5C2B3D2B3D9F7D2B70000C2B765
:100C410022C2B2D2B27908C2A6A2B633D2A6D9F7CD
:100C5100F56322C2B2D2B27908C2A6A2B033D2A63B
:100C6100D9F7D2E6D2E7F56422E56330E603C2079D
:100C71002220070AE552041207AAF552D20722E5FB
:100C81006430E103C2082220080AE552041207AACF
:100C9100F552D20822E56330E103C2092220090D91
:100CA1000565E5651206FCF565D205D20922E56404
:100CB10030E503C20D22200D06B202D203D20D226D
:100CC100E56330E203C20A22200A06B200D205D24D
:100CD1000A22E56330E703C20B22200B0D1567E5FD
:100CE10067120717F567D205D20B22E56430E403DA
:100CF100C20C22200C0D0567E56712070EF567D2BD
:0E0D010005D20C22E56430E303C21F22201F3E
:100D0F0006D21F120D2E2222E56330E011E564207A
:100D1F00E003C22022202006D220120D2E222230E4
:100D2F001603D21922D20322301409E55FD2E1D281
:100D3F00E2F55F22E552B40009E55FC2E1D2E2F5C8
:100D4F005F22B40109E55FC2E2D2E1F55F22B4028E
:100D5F0009E55FC2E2C2E1F55F22E55FD2E2D2E1CF
:100D6F00F55F22E55FD2E3D2E4D2E5F55F30050708
:100D7F00120DA330040122E565B40007E55FC2E35D
:100D8F00F55F22B40107E55FC2E4F55F22E55FC2BC
:100D9F00E5F55F22E565B5660122E566B40007E576
:100DAF005FC2E3F55F22B40107E55FC2E4F55F229E
:100DBF00E55FC2E5F55F22200207E55FD2E7F55F49
:100DCF0022E55FC2E7F55F22E55FD2E0D2E6F55F8D
:100DDF00300507120DFA30040122200007E55FC22B
:100DEF00E6F55F22E55FC2E0F55F2220010A3000E1
:100DFF0010E55FC2E6F55F22200006E55FC2E0F571
:100E0F005F22755DFF755EFF300507120EC030045F
:100E1F000122E567B40007E55DC2E0F55D22B4018C
:100E2F0007E55DC2E1F55D22B40207E55DC2E2F5BB
:100E3F005D22B40307E55DC2E3F55D22B40407E567
:100E4F005DC2E4F55D22B40507E55DC2E5F55D22FF
:100E5F00B40607E55DC2E6F55D22B40707E55DC29E
:100E6F00E7F55D22B40807E55EC2E0F55E22B4093E
:100E7F0007E55EC2E1F55E22B40A07E55EC2E2F560
:100E8F005E22B40B07E55EC2E3F55E22B40C07E504
:100E9F005EC2E4F55E22B40D07E55EC2E5F55E22A3
:100EAF00B40E07E55EC2E6F55E22E55EC2E7F55ECB
:100EBF0022E567B5680122E568B40007E55DC2E089
:100ECF00F55D22B40107E55DC2E1F55D22B40207CD
:100EDF00E55DC2E2F55D22B40307E55DC2E3F55DB2
:100EEF0022B40407E55DC2E4F55D22B40507E55DB4
:100EFF00C2E5F55D22B40607E55DC2E6F55D22B4F5
:100F0F000707E55DC2E7F55D22B40807E55EC2E0BD
:100F1F00F55E22B40907E55EC2E1F55E22B40A0769
:100F2F00E55EC2E2F55E22B40B07E55EC2E3F55E55
:100F3F0022B40C07E55EC2E4F55E22B40D07E55E50
:100F4F00C2E5F55E22B40E07E55EC2E6F55E22E568
:100F5F005EC2E7F55E22E56C75F003A4900F6F7328
:100F6F0002102F02103402103902104102104602F3
:100F7F00104D02105402105E02106502106C021028
:100F8F007302107DE56C75F003A4900F9D73021032
:100F9F002F0210340210390210410210390210349E
:100FAF00E56C75F003A4900FB97302102F02103483
:100FBF0002103902104102104602104D0210540265
:100FCF00105E02105402104D021046021041021022
:100FDF0039021034E56C75F003A4900FED73021015
:100FEF002F02103402103902104102104602104D28
:100FFF0002105402105E02106502106C0210730290
:10100F00107D02107302106C02106502105E021048
:10101F005402104D021046021041021039021034D2
:10102F00E54D021084E54E021084E54F12142A029A
:10103F001084E550021084E54D240C021084E54E17
:10104F00240C021084E54F240C12142A021084E59C
:10105F0050240C021084E54D2418021084E54E2410
:10106F0018021084E54F241812142A021084E55038
:10107F002418021084F5421205371204F622E56493
:10108F0030E203C20E22200E10D20E2014041210D2
:10109F00A9221205371204F62222E552B4000B05DD
:1010AF006C120720F56C120F6522B4010B156C1230
:1010BF00073FF56C120F6522B40208056CE56C1240
:1010CF00076922E551B4000A12086575F055021040
:1010DF00F422B40C0A12086575F0240210F42212DF
:1010EF00086575F01784F56C120F6522E56430E31F
:1010FF000320E009200605756C03D20622C20622E2
:10110F001203EB853630853731120407B42F0302F3
:10111F0011235010C21475F00C8412070575F00CD2
:10112F00A4F55122D21475F00C84C3940385F07387
:10113F0075F00CA4F56D12187E2553256DF542221E
:10114F00120397853C82853D8312037875F01784CF
:10115F00F553B5540122F554D20322F555B5560176
:10116F0022F556D20322E56320E4077558181211B1
:10117F009B2230E50775580C12119B2275580012EF
:10118F00119B22FFE56D75F00CA42F22E558B55782
:10119F000122F557D203221203B3853A30853B3132
:1011AF007532007533007830753400753500793439
:1011BF001202958682088683858230858331753247
:1011CF00007533007830753422753500793412028A
:1011DF00C0E61203B3853A30853B31120407F97527
:1011EF00F00C8485F055120853F56DE55512116A10
:1011FF0012120612114F22E9B56E0122F56ED203BB
:10120F00221203B3E567B40F03021247121290EDD7
:10121F00932558F53EF54DA3ED932558F53FF54E23
:10122F00A3ED93121431F540F54FA3ED932558F527
:10123F0041F5502212124B221213CE22300004120B
:10124F0012762212125622121290ED932558F53E65
:10125F00A3ED932558F53FA3ED93121431F540A359
:10126F00ED932558F54122121290ED93F53EA3ED23
:10127F0093F53FA3ED93121438F540A3ED93F54189
:10128F0022E56775F00CA4FD2000069009D202122A
:10129F00A3900A92E565B4000122B4010679041205
:1012AF0012B82279081212B822A3D9FD22E56320C1
:0E12BF00E0041212EB2230E3041212EB2212B2
:1012CD0012EB22E56320E008C216757100D22622CA
:1012DD0030E308302604C226C21822D22622E56742
:1012ED00B40F10200008E565B40252021300E56545
:1012FD00B4024A121290ED932555F54D25532558FC
:10130D00121192F53EA3ED932555F54E2553255813
:10131D00121192F53FA3ED932555F54F2553255801
:10132D0012119212142AF540A3ED932555F550256F
:10133D00532558121192F54122121441221213CE47
:10134D0022E56430E30630E003C20F22200F15D2F0
:10135D000FE567B40F0E200006E565B4023522E5F2
:10136D0065B4020122E5657015120923FC120923EB
:10137D00FB120923FA79009000191213DF221209CA
:10138D0044FC120944FB120944FA79009000191229
:10139D0013DF22E56570151208F6FC1208F6FB1234
:1013AD0008F6FA79009000151213DF2212091DFCC0
:1013BD0012091DFB12091DFA79009000151213DF99
:1013CD00223000079000191213EB22900015121312
:1013DD00EB22E9F0A3EAF0A3EBF0A3ECF022E02579
:1013ED0055F54D25532558121192F53EA3E025557F
:1013FD00F54E25532558121192F53FA3E02555F5CD
:10140D004F2553255812119212142AF540A3E025A9
:10141D0055F55025532558121192F5412220020100
:10142D0022240C2220020325582222200203240C00
:10143D002224002230000412147C2212144C221299
:10144D001290ED9325532558F53EF54DA3ED9325BB
:10145D00532558F53FF54EA3ED932553121431F551
:10146D0040F54FA3ED9325532558F541F550221224
:10147D001290ED932553F53EA3ED932553F53FA320
:10148D00ED932553121438F540A3ED932553F541F3
:10149D00221203CF853830853931120407C3B46F5A
:1014AD000DD216201807D219757100D218224003DB
:1014BD000214AED217C218C216B56A0122F56A120D
:1014CD00151AF569B56706E566B5650622F567D2A5
:1014DD000522F566D2052275F00C84A8F075F0048E
:1014ED00A4F9E875F00384AAF012150829B40F03C6
:1014FD00C2002240FBC39410D20022BA00047565CD
:10150D000022BA01047565012275650222F8B43C0A
:10151D0003021523500412152B2212153722793C84
:10152D00C9C3991207EF1214E422C3943D2430125B
:10153D0007DD1214E4227587907589227598507510
:10154D008C38758A38C0D043D00878197C0A7D0A4A
:10155D00D0D0D28CD2A9D2AF22C0E0C0D043D00817
:10156D00DD177D0AD8137819B210D904A972D215D6
:10157D00DC077C05300502B204D0D0D0E032121564
:10158D00B912114F20100F121681121612121629B0
:10159D0012186A1216AA1216911216401216BB12C2
:1015AD000C001217A212172012176A22120C4212E7
:1015BD000C54E56420E316C212756700121C091263
:1015CD000C42120C54E56420E3040215CC222212C5
:0715DD000C42120C54E564FE
:1015E40020E30FE56330E20122201309D21375676B
:1015F4000022C21322120C42120C54E56430E3F5AB
:10160400C213D212121C19740090001DF022E5635B
:1016140030E103C2092220090B90001DE0041208E6
:1016240041F0D20922E56330E603C2072220070B0A
:1016340090001DE01412084AF0D20722E55FD2E1BF
:10164400D2E2D2E3D2E4D2E5F55F90001DE0B4002B
:1016540007E55FC2E1F55F22B40107E55FC2E2F589
:101664005F22B40207E55FC2E3F55F22B40307E536
:101674005FC2E4F55F22E55FC2E5F55F22E5633012
:10168400E203C20A22200A04B211D20A22E55FD27E
:10169400E0D2E6F55F201107E55FC2E6F55F22E5DB
:1016A4005FC2E0F55F222011071217C41217DB2274
:1016B4001217F91218102220110D755DFF755EFFC7
:1016C4001217F2120E2122755DFF755EFF121827A4
:1016D400120E212290001DE0B4000490001E22B4DA
:1016E400010490001F22B4020490002022B40304D9
:1016F400900021229000222290001DE0B40004906A
:10170400002322B4010490002422B4020490002592
:1017140022B403049000262290002722E558255382
:10172400F5307531007532007533007830858234B8
:1017340085833579341202B075340A7535007934ED
:101744001202C01216FCE0F5347535007934120229
:101754009575340775350079341202A2868208869D
:1017640083AE82AF832290001DE0B400088E438FC5
:10177400441204C922B401088E458F4612049C22E7
:10178400B402088E478F4812044222B403088E49DB
:101794008F4A12046F228E4B8F4C1204F6221216BB
:1017A400D8E0F53075310075320075330078307546
:1017B400345775350179341202958682088683225E
:1017C400E56330E703C20B22200B0B1216D8E0149A
:1017D400120717F0D20B22E56430E403C20C222076
:1017E4000C0B1216D8E00412070EF0D20C221216BB
:1017F400D8E0F56722E56330E703C20B22200B0B28
:101804001216FCE014120717F0D20B22E56430E440
:1018140003C20C22200C0B1216FCE00412070EF07B
:10182400D20C221216FCE0F56722E56320E404756D
:1018340058242230E5047558182275580C22E563A3
:1018440020E4047558482230E50475583C22755844
:101854003022E56320E40475586C2230E5047558A1
:10186400602275585422E56320E00412182E2230B9
:10187400E30412184222121856227A00856F8285D8
:101884007083EA93B46302EB22B573012240012210
:101894000AFB021886E56775F005A4F920000D908F
:1018A4000B521218BD85826F85837022900BA9128A
:1018B40018BD85826F85837022700122A3D9FD2211
:1018C40020160475710022201C0905711218E212F9
:0718D400190622C21C157168
:1018DB001218F91219062290003BE0B571047571CC
:1018EB000122E571B411047571012250FA22E571E0
:1018FB00B4000790003BE014F57122A97190002A07
:10190B00E5716007A3D9FD12191D2290002B121946
:10191B001D22E0121931F9540FF567E9C4540FC2B7
:10192B00E3FA1215082220E703C20022D20022E5B7
:10193B006330E703C21D22201D08D21CD219D21717
:10194B00D21D22E56430E403C21E22201E06D219EA
:10195B00D217D21E2212199912114F121175201083
:10196B000BC2051219ED121A40120CAF121AB0125B
:10197B001AC3121AE7120DC6120C001212BC120572
:10198B002312044212046F12049C1204C922120C7B
:10199B0042120C54E56420E313C21A121C29120CD8
:1019AB0042120C54E56420E3040219A92222120C02
:1019BB0054E56420E30D30E40122201B09D21B7592
:1019CB00670022C21B22120C54E56430E3F8C21BE1
:1019DB00D21A121C39740090003CF090002B121993
:1019EB001D22E56330E603C22522D2251219FE1211
:1019FB001A1F22E56330E703C22122202115D221D1
:101A0B0090003CE0141207C5F0B4100122121A75B5
:101A1B0012191D22E56430E403C22222202215D2C2
:101A2B002290003CE0041207BCF0B4100122121A01
:101A3B007512191D223025012290003CE0B41007CD
:101A4B00121A82121A9922120C96120CC1120CD372
:101A5B00120CEC121A6222E565C4F9E567693000D5
:101A6B0002D2E7F8121A75E8F02290003CE004F974
:101A7B0090002AA3D9FD22E56330E703C22322207D
:101A8B00230B90003BE0141207D7F0D22322E5641E
:101A9B0030E403C2242220240B90003BE004120705
:101AAB00CEF0D2242290003CE0B410067402120D4A
:101ABB0045227403120D45222025012290003CE0A3
:101ACB00755DFF755EFFB4100122120E23E55FD228
:101ADB00E3D2E4D2E5D2E0D2E6F55F223025012253
:101AEB0090003CE0B4101E90003BE01414755DFFB9
:101AFB00755EFF120E23E55FD2E3D2E4D2E5D2E0AE
:101B0B00D2E6F55F22120D72120DD7120E1122E0E2
:101B1B00A343D20205A2F0A375D25275D2A2C2156D
:101B2B00757204201505E5D220E0F853D2FD05A20D
:101B3B00D9DD2243D202438E20E0A353D2FD538E34
:101B4B00DF05A2F0A305A2D9EA22790A7407900057
:101B5B001EF0A3D9FC121C0922740290003BF074F6
:101B6B001F90002BF0741F90002CF0741F90002D11
:101B7B00F0741F90002EF0741F90002FF0741F90C4
:101B8B000030F0741F900031F0741F900032F0742D
:101B9B001F900033F0741F900034F0741F900035C9
:101BAB00F0741F900036F0741F900037F0741F9084
:101BBB000038F0741F900039F0741F90003AF01247
:101BCB001C2922120C54E56430E30122121B55121E
:101BDB001B64C212C21AE55FB2E0B2E6F55F120CEB
:101BEB0000120281120281120C54E56430E3E712F9
:101BFB00028CE55FD2E0D2E6F55F120C0022790A87
:101C0B0090001E05A290000005A2121B1A22790A51
:101C1B0090000005A290001E05A2121B3E22791116
:101C2B0090002B05A290000A05A2121B1A22791113
:0E1C3B0090000A05A290002B05A2121B3E226B
:00000001FF
